:03000000020030CB
:03001B000200A838
:10003000759000758921758800758160758CFA75D9
:100040008A24758DE7758BE775A888D28E7F007539
:1000500032007533147E1475310020B2FD20B20ACF
:10006000758CFA758A24C28D015DD28C20B2FDC2D6
:100070008CE58CC20030E70AD200F4F58CE58AF4F6
:10008000F58AE58C13E58A13F5301200CFF532704E
:10009000067531000200A62000067531010200A697
:1000A0007531020200A6015DC0E0C0D0EF60061FFE
:1000B000DF03752100DE0DAE33E532FF75210370DD
:1000C00003752100E5315521F590D0D0D0E0329074
:1000D00000D4932200000000000000000000000097
:1000E0000000000000000000000000000000000010
:1000F00000000000000000000000000001010101FC
:1001000001010101020202020202020203030303CF
:10011000030303030404040404040404050505059F
:10012000050505050606060606060606070707076F
:10013000070707070808080808080808090909093F
:10014000090909090A0A0A0A0A0A0A0A0B0B0B0B0F
:100150000B0B0B0B0C0C0C0C0C0C0C0C0D0D0D0DDF
:100160000D0D0D0D0E0E0E0E0E0E0E0E0F0F0F0FAF
:100170000F0F0F0F1010101010101010111111117F
:10018000111111111212121212121212131313134F
:10019000131313131414141414141414151515151F
:1001A00015151515151515151515151515151515FF
:1001B00015151515151515151515151515151515EF
:1001C00015151515151515151515151515151515DF
:0401D00015151515D7
:00000001FF
